:020000040000fa
:08000000e40804000000000008
:020000040000fa
:10040000889fbe008a9fbe00010578000100e000c1
:100410000400350008003c000000e000200032002d
:100420000500370060001000e080180002003b006b
:1004300001f02c001a0037000004be006011b80063
:100440006b0920000982cf00020039000882cf002a
:100450000441b000694252000e00320008003b0027
:1004600082817100610164008904d1000884d30095
:100470008b05e8000442e800f9ff3a000500370068
:100480000804440089844c008b05e9000442e9001b
:10049000fbff3a00540107000af0a70001f0a0009a
:1004a0004f05be004f04be0000000600889fbe003e
:1004b0008a9fbe008c1f780071010700780133000d
:1004c00003866c006450e100240032006420e100e7
:1004d000270032006150e100220032006120e1007b
:1004e000210032008b854200eb07b1000134b800d7
:1004f000003ab8000804420089844a00013ab80072
:100500000030b8008880400009014a000400330030
:100510000000400081804800020149008b05e9008d
:10052000c909dd00830170000100320013002000c2
:10053000c814de004814dd004709de001200b200d6
:10054000c808de00088470002701070001f0a10040
:100550000cf0a70001f0a0005a0137006120e10073
:100560005c0132000801be000200be00f7ff370048
:100570006150e100fcff3a0056013700889fbe0041
:100580008a9fbe008c1f78003d01070044013300a4
:1005900003866c006450e1002e0032006420e1000c
:1005a000330032006150e1002f0032006120e10091
:1005b0003100320085855500eb07b00009002000ae
:1005c00008042000050037000804440089844c001a
:1005d0000a0031000603430087834b0000015300eb
:1005e00081815b00f8ff33000203be000800a00019
:1005f0000804440089844c00f6ff3900c639dd0048
:100600008301730001003200130020008904d1002f
:100610000884d3000998a300050032000800a70051
:100620000300a0008904d1000884d3008b05e800f2
:100630008904d1000884d3000001eb000281d200bc
:10064000e900070001f0a1000cf0a70001f0a000f4
:100650001c0137006420e1001e0132000801be00c9
:100660000200be00f7ff37006120e10019013200ef
:100670006000b800f3ff37000000200001f82700f9
:10068000f0ff370003f0a200889fbe008a9fbe00e3
:100690008c1f7800fa000700010133006450e1006c
:1006a0004f0032006420e1005200320003826c00ef
:1006b00007003b000905d0000306d000820f54005c
:1006c0000c065d000200390002003200890178004a
:1006d000030678008582550004003d000003fd00fc
:1006e0008103fd008502ea008b854200840f7200c1
:1006f00002003b0060001000e08018006011b800ac
:100700000005eb007a28e1000a00390006007800b5
:10071000c75ddd00f707b200878075002d00370048
:10072000828171000a017800610560008180d1003a
:100730000080d3008502e900f9ff3b000604400079
:100740008784480002003b0060041400e0841c0021
:100750000988a300070032008a817100828171003c
:10076000610164008904d1000884d3008b05e8008e
:10077000170037000978a30013003a000b00e000cf
:10078000130034008b05e9000804440089844c0000
:100790000a4474000978a3000d003a000b00e00041
:1007a000070034008b05e9000804440089844c00ec
:1007b00001003a000b0020000978a300f7ff320087
:1007c0000001eb0002003700828171000a0178000d
:1007d000850007000cf0a70001f0a000b900370069
:1007e0006420e10002003a00838f6c00b9003300fe
:1007f0000801be000200be00b20037000001be00ca
:10080000b70007000470a70003f0a1006509b1005c
:10081000160032000d0035006828e10006003500a2
:10082000f0ff2f00f1ff27000300e00013003b0062
:100830000100280000000500000040008180480001
:100840008502e900fcff3a0008003700f88f4200fb
:1008500002003c008000eb00000005008100d10098
:100860000080d3008502e800fcff3a000300e000ae
:1008700002003b0060001000e0801800000006004d
:10088000889fbe008a9fbe008c1f78007c000700f6
:100890001002200002003b0000408800800037006a
:1008a0008a0062006408e10002003a00004088000b
:1008b000880037006108e100fcff32000800be003c
:1008c000030478002dff070001f0a1009900070044
:1008d00008f0a600040037000001be0091042400c7
:1008e000b0fd200067ff070009f0a70001f0a2009b
:1008f00074003700889fbe008a9fbe008c1f78005e
:100900000004be00760007000478a30026003a0029
:100910006120e1002500320009f8a30025003a001b
:100920006420e10021003200f507b1000508a300b2
:100930000200320000004000818048006044b8009e
:1009400003102000020020000000400081804800c9
:100950000805440089854c000a0541008b85490043
:100960000a0550008b855800030033000a00be00c2
:1009700002047400838474008301d1000281d300d7
:10098000830f7100f0ff3a008904d1000884d3007e
:100990006001490082017800c1adde00fb07b000b4
:1009a00011000700470037000960a0000800be00e2
:1009b000440037001202200002408800f0ff2f00a0
:1009c000f1ff27003f0037000001eb00be003700b9
:1009d0000081eb00bc0037000001eb002301370071
:1009e0003200200021013700810020006180550085
:1009f0000b003d000b00200061fe2f000100e10014
:100a00001d00340082817100610164008904d100fd
:100a10000884d3000000e800faff3a0071002000cb
:100a200061006400030070000200600009003200f1
:100a300061044400e0844c000988a50005003200f0
:100a40008b05e8006808e10002003a008904d10043
:100a50000884d300f20f20000258e10005003d0099
:100a6000c75ddd00f907b2008980750008007800d5
:100a7000000006000bf827008b007800000005003e
:100a80000004be00160007000003be000405be00ff
:100a90000200be0012000700844f7500000006002f
:100aa0000200be006450e100050036006420e10051
:100ab000020036000968a30001003a000800be00e9
:100ac0000160a0004f0678004f05be004f04be0035
:100ad00000000600f0ff2f00f1ff2700f9ff3700ac
:100ae000c70ade00f107b200f50fb20008003200bd
:100af000e1cf4200020032000170a0002400050096
:100b0000810f700001003200040805004400050058
:100b1000810f700002003a00140005008502e90010
:100b20000000400081c04800fcff3b000170a000b5
:100b300024000500889fbe008a9fbe008c9fbe00d7
:100b40000004be00e6ff07000800be00890678002a
:100b50006420e10008003900040032000160a000b8
:100b600012022000024088005300370091fc23004d
:100b7000b0fd20004e0037000006eb0009f0a10098
:100b800003f82300020020000800be001e01070039
:100b90000600340001f82300000020000801be0018
:100ba00076fe07000004be002c0020000800be00f6
:100bb00093e82300320a23001301070012003400d7
:100bc0000801be00d1fd2300703d2b00aefe0700e2
:100bd0000005be00b3f32300f27a26000800be0031
:100be00032fe070003f8230002002000a5fe0700e4
:100bf0000801be00a4fe07000a01be005ffe070058
:100c00000004be000c06e8000800be0001f0a100d0
:100c10000200200003982300fb0007000800be002c
:100c2000160035000801be0020fe07000005be00ca
:100c300032cd2c0043fb230093fe0700809fbe00b3
:100c40001269280003d52b000a00be0017fe07001a
:100c5000620f210013ef2b008bfe07000a01be007c
:100c600012fe07004f01be0044fe07000801be004f
:100c70000efe07000801be0083fe07000c00e00026
:100c80000b0032000c10a70001f0a200b2fd200002
:100c900093fc23006260e1000400320022a92000de
:100ca00063f023000c10a70063f8230076fe070012
:100cb0000df0a70001f0a2004f06be004f05be00d8
:100cc0004f04be0000000600889fbe008a9fbe0041
:100cd0008c9fbe00820578000004be0080ff0700e4
:100ce0000800be006420e1000700390002003a005d
:100cf000f1ff2700f0ff2f000160a000120220008a
:100d000002408800550037006120e10003003a00ee
:100d10000b00a70001f823005000370001f0a100ec
:100d20000200210093642400b70007000800be0001
:100d300004003500b2fd2000930c2400b40007002d
:100d40000004be000005eb000b00a6004f0dde0006
:100d500001f0a1000004be0032982f0023ea230016
:100d6000d2fd07000001eb0003f023000b00a700f9
:100d700003f8230044fe0700a0fe07000000a700c0
:100d80000a00a2009efd07000b00e00003003200f5
:100d90000200200003f023003afe070001f0a20049
:100da0000006be000200200093042400bffd0700df
:100db0000801be0034fe0700809fbe000c00be008c
:100dc00022a22a00d3a72300b8fd07004f01be00ce
:100dd0002dfe07000004be0001f0a100020020006b
:100de00003982300880007000800be0019003500a2
:100df0000001be00adfd07000006be00b2c529001f
:100e0000e3622300a9fd070022222b00f3942b00ac
:100e10001dfe07000c01be00a4fd0700e2732800c0
:100e200083c0230018fe07000c01be009ffd0700d1
:100e300042aa2a00a3e22b0013fe07000c01be0009
:100e40009afd07000801be0098fd07000801be00da
:100e50000dfe07000a00a70001f0a2004f06be0029
:100e60004f05be004f04be0000000600889fbe0074
:100e70008a9fbe008c9fbe000206780001f0a7008a
:100e80000cf0a0000004be0015ff07000800be0023
:100e90006420e1000700390002003a00f1ff27005a
:100ea000f0ff2f000160a000120220000240880025
:100eb0005100370009f0a1000800be000200200028
:100ec00003f8230054000700f4ff3c000800be00b4
:100ed00002002000039823004b0007000800be001a
:100ee000300035000200200003f023004a00070014
:100ef00005003c000800be000801be006bfd0700b5
:100f00000005be000e0037000c10a20000002000fb
:100f100001f823000801be00dafd070002002000ee
:100f200003f0230061fd07000005be0071fe07000d
:100f30000200200003002c005cfd07000004be003e
:100f40000a00be00b2d02800130b2c00cefd070013
:100f50000a01be0055fd0700020f2500330b2400d7
:100f6000c9fd0700809fbe000a00be005206220095
:100f700013f02b004dfd0700b2662100f3f62300ad
:100f8000c1fd07000a01be0048fd07004f01be0079
:100f90007afd07000801be0044fd07000801be00fd
:100fa000b9fd07000c00a70007003700b2fd2000c4
:100fb00093fc23000c10a700b3fd07000cf0a70062
:100fc00001f0a2000c0037000cf0a700020037006f
:100fd00001f0a20004003700b2fd200093042400b9
:100fe0000c10a60003003700b2fd200093fc230084
:100ff0000c10a700a4fd07004f06be004f05be0061
:101000004f04be000000060014002000040037005a
:10101000040020001d003700f4ff2f0000003700ff
:10102000889fbe008a9fbe00841f780094fe070040
:101030004f00780011003300f0ff2f00838f6c0009
:1010400006003b00040565000a00a7000800370001
:1010500009f0a6001000200008003700820f54009d
:10106000838f5c00030039001000200001003e0067
:101070000000200009f0a7000000ea004f05be00b4
:101080004f04be000000e00000000600889fbe0084
:101090008a9fbe008c1f78004f26dd0078fe070077
:1010a0007ffe33006120e100430032006250e10026
:1010b00041003e003e0039006420e1003c00320067
:1010c000058255000f003b000402e80038003a009a
:1010d000800f5300818f5b00350034000800be0094
:1010e00003f0a10001f0a60003f0a0000cf0a7009f
:1010f00065fd070073fe37000603430087834b003e
:101100000c4646000005530081855b000200330059
:101110000a03be000c00a0000402e900f6ff3b0039
:10112000850578000602430087824b0004003a00e0
:101130006000b80009f0a70001f0a00061fe3700d0
:101140000002520081825a000704e00004003300cc
:101150000603430087834b008b05e900faff370045
:10116000090578000604be000203be006011b80045
:101170001dfe0700e00f5200e08f5a000700350007
:1011800002003c000c08a300040032000601be006f
:1011900003f0a0000cf0a7003bfd07000a856800e3
:1011a00001f0a1000af0a70001f0a00045fe370001
:1011b0000800be0043fe3700100220000cf0a6001d
:1011c0000040880043fe37008fe22000007f2400ab
:1011d0000001880000000000340f02000000000041
:1011e000e0012000303a880044e7a90044c7a90084
:1011f0004487a9004467a9004447a9004427a900df
:101200004407a9003000200031742000820720002c
:10121000a30920008248780083487800804878003d
:1012200010002000217420006204200073052000bb
:101230008248780083487800804878002aa3ef002d
:101240002c23ef002023ef0021e3a90021a3a80015
:101250002183a8002143a8002123a9002103a9007c
:1012600020e3a80020c3a80020a3a8002063a900b1
:101270002043a9002023a90023e3a90023c3a90038
:1012800023a3a9002383a9002343a8002323a900a3
:101290002303a90022a3a8002283a9002263a80097
:1012a0002243a8002223a9002203a900f0f1210073
:1012b000201988003223ef002623ef002823ef00b7
:1012c00029e3a90028e3a9002963a9002943a9006b
:1012d0002923a9002903a9002863a9002843a900fc
:1012e0002823a9002803a9002e23ef00f0ff2000e7
:1012f00080198800aa80a900aaa0a900aac0a900f4
:101300008ca3a9008c83a9008c23a8008c03a900be
:10131000d0c0b300701c88009023ef00c0022000f2
:10132000901c880000302000a01c8800b000200025
:10133000b01c8800ab40a900ab20a900ab00a900fd
:1013400085c0a90000002000401188002222ef0083
:1013500023e2a90023a2a9002022ef002042a80036
:101360002022a9009580a9009560a90030102000d6
:10137000c011880033e2a90033a2a900b340a8003d
:10138000b320a900b300a9003022ef003042a90029
:101390003022a90032e2a90032c2a90097e0a900d8
:1013a00097c0a900a4c0a800a4a0a900a480a80078
:1013b0004221ef0010082000100a8800a6c0a800f3
:1013c000a6a0a900a680a8004621ef0010082000d2
:1013d000300a8800b6c0a800b6a0a900b680a80050
:1013e0004a21ef0010082000500a8800b740a800ea
:1013f000b720a900b700a8004e21ef001008200078
:10140000700a8800b7c0a800b7a0a900b780a800dc
:101410005221ef0010082000900a8800b840a80070
:10142000b820a900b800a8005621ef002000200035
:10143000b00a8800a540a800a520a800a500a90022
:101440008421ef00a740a800a720a800a700a900ba
:101450008a21ef00b0c0a800b0a0a800b080a90009
:101460009021ef00b140a800b120a800b100a90070
:101470009621ef000622ef000822ef00ca22ef00bb
:10148000d022ef00d622ef00e222ef00c6a2ef004a
:10149000cca2ef00d2a2ef00dea2ef00cdc2a900e5
:1014a000cda2a900d202a900d222a900d242a9004d
:1014b000d262a900de02a900de22a9001e21ef00ef
:1014c0002021ef001421ef001821ef003000200050
:1014d000e008880000d42000d00888001e61a80021
:1014e000b240a900b220a800b200a8008780a900dd
:1014f0009780a8001021ef000621ef00400d230087
:101500006008880010a1a80084e0a90094e0a80069
:10151000a7c0a800a7a0a800a780a9001221ef00db
:101520000a21ef00f0ff2f00700888001281a80048
:101530002c21ef002221ef0090d0230040098800e9
:101540002c81a8002ca1a800bbc0a800bba0a800ab
:10155000bb80a90089e0a90099e0a8002e21ef0036
:101560002621ef0090d02300500988002ea1a8006a
:101570002e81a800bc40a800bc20a800bc00a90087
:101580008a00a9009a00a800a440a900a420a800ed
:10159000a400a9008200a9008400a9009400a8006a
:1015a0000421ef000021ef0005e1a900da0c0200a0
:1015b00000000000704f24001056880000002e002c
:1015c00020568800704f24003056880000002e00fe
:1015d00040568800704f24003047880000002e00dd
:1015e0004047880021e2a800ce0c02000000000065
:1015f00080c02000b05a88008560a90021e2a800c0
:1016000087c0a90097c0a80031e2a8008900a900fe
:101610009900a8008420a9009420a80084a0a90013
:1016200094a0a80088a0a90098a0a80088c0a9003c
:1016300098c0a80088e0a90098e0a8008440a9000c
:101640009440a80084c0a90094c0a8008720a900e5
:101650009720a8008740a9009740a800e202a900af
:10166000e222a90085a0a90011e1a8002de1a800af
:10167000a03a2000f0478800100c88004075200038
:101680000048880030a0200010488800c0da200000
:101690002048880054380200000000000b08a90010
:1016a0001009a90010a9a9001069a9000c28ef00d1
:1016b000b04a8000030120000300b9004306200067
:1016c000110009004308d80080508800204980009c
:1016d000030120000300b9004306200011000900a7
:1016e0004308d800405088003049800003012000a2
:1016f0000300b90043062000110009004308d80088
:101700005050880040498000030120000300b900c8
:1017100043062000110009004308d80060508800eb
:1017200050498000030120000300b9004306200057
:10173000110009004308d80070508800204a80003a
:10174000804b8800030120000300b90043062000fd
:10175000110009004308d80010508800304a80006a
:10176000030120000300b900430620001100090016
:101770004308d80030508800404a80000301200010
:101780000300b90043062000110009004308d800f7
:1017900020508800b0498000b04b88000301200031
:1017a0000300b90043062000110009004308d800d7
:1017b000005088008000eb00804980000002020099
:1017c00000000000d1528800e05288008000eb0049
:1017d000a0498000000202000000000011538800b0
:1017e000205388008000eb00f049800000020200d6
:1017f000000000000312240002002000be020200cc
:101800000000000031538800405388008000eb0046
:10181000104a80000002020000000000715388009e
:10182000805388008000eb00904980000002020095
:1018300000000000f1528800005388008000eb0097
:10184000004a80000002020000000000515388009e
:10185000605388008000eb00e04980000002020035
:1018600000000000e14f8800f04f88008000eb008e
:10187000d049800000020200000000000312240092
:10188000020020005602020000000000f15788000c
:1018900000588800414b8000304b8000000202005d
:1018a00000000000a3c52400920e2900be02020021
:1018b00000000000a14c8800904c8800434b800041
:1018c000324b8000660e020000000000819a20006a
:1018d000e0b42000a0107800a0107800a0107800dc
:1018e000a0107800a0107800a0107800a010780058
:1018f000a0107800ac09a9003a0baf00ac09a80011
:10190000614b8000504b800000020200000000008c
:10191000a3c52400920e2900be02020000000000b0
:10192000c14c8800b04c8800634b8000524b800053
:10193000660e020000000000e19b2000e0b42000e1
:10194000a0107800a0107800a0107800a0107800f7
:10195000a0107800a0107800a0107800a0107800e7
:10196000a0107800c009a9003a0baf00c009a80078
:101970000689a90038e9af000689a80006a9a900d0
:101980003909af0006a9a80021e3a8008de3a8004b
:101990002043a80000000000feff37002e2aef00c1
:1019a0002c2aef002a2aef001fe1a80013e1a8006b
:1019b000000006002180200062e220008018eb0079
:1019c0000208e600fdff3700000006009246800096
:1019d0000290b9007059880081598800a2468000a1
:1019e0000290b9002e2bb4000100780030abb40097
:1019f000b24680000290b9002e2bb400010078009e
:101a000030abb4001a0e02000000000070598000d4
:101a1000005288000000060090468000105988009f
:101a2000a24680000290b900705988008159880050
:101a3000b24680000290b9002e2bb400010078005d
:101a400030abb4001a0e0200000000007059800094
:101a500000598800b146800001f0a700202bee005d
:101a6000005980008000eb0000f0a7008080eb00b0
:101a70000002020000000000d1568800e0568800f5
:101a8000105980008000eb0000f0a7008080eb0080
:101a90000002020000000000d3568000e2568000e1
:101aa000400402000000000091548800a054880007
:101ab00000000600a0468000105988009246800071
:101ac0000290b9007059880081598800b2468000a0
:101ad0000290b9002e2bb4000100780030abb400a6
:101ae0001a0e0200000000007059800000598800a2
:101af000b146800001f0a700202bee0000598000c5
:101b00008000eb0000f0a7008080eb0000020200e4
:101b100000000000d1568800e0568800105980006f
:101b20008000eb0000f0a7008080eb0000020200c4
:101b300000000000d3568000e256800040040200fe
:101b400000000000b1548800c05488000000060066
:101b500012598000f30720000310b90004598000d7
:101b6000110009004408d800705988002febaf001d
:101b70002e2bee00f10320002159880000002000e8
:101b800090018800c0922300215980004200a900e2
:101b90008180d200008040009000ba00725980001d
:101ba0000208e60002003700242bed00f3ff3a00a4
:101bb000240be20018003200d7e8ae00070037001f
:101bc00023ebae000c0037000008200021598000f4
:101bd00001004000305988000000060023ebae00f1
:101be0000a00370000102000215980000100500039
:101bf00030598800000006000008200021598000ac
:101c00000100500030598800000006002059800073
:101c10003059880000000600d7e8af000200370006
:101c2000262bef0000000600000820003059880035
:101c300000000600308bd6004200af000000060016
:101c4000d00e020000000000da0e020000000000ca
:101c5000000120005059880036abd60038abd600c2
:101c600032abd60034abd60036abd60038abd6009c
:101c700032abd60034abd6004200a8002eabd60063
:101c800030abd60080598000340bb50002003a001a
:101c900070598000320bb500050039007059800082
:101ca000322bb5008059800034abb5002e2ba80034
:101cb0002e0ba9002a2bed00e7ff3a004200a900f5
:101cc00030abd7002eabd70000000600282bef006a
:101cd000e40e0200000000004200af000000060019
:101ce0001c0f020000000000000220005059880074
:101cf0000281d2008381d200e6b4200009000800ee
:101d000006000000168bd200a0002000960078008c
:101d1000008050004200af00000b780026007800e1
:101d20002a2bed00f2ff3a00280baf003a0ba80077
:101d30004200a9000000060040598800000220006f
:101d400050598800c2b32000a00020004200a90022
:101d50004159800001800800020000004200af00ed
:101d6000120940001299d30030abd7002eabd70038
:101d70002a2bed00f3ff3a0042007800f1ff2f001c
:101d8000008040004200ae00308bd6004200af0021
:101d9000000006003a0baf000e000700000006002e
:101da00070598000b059880080598000c05988005f
:101db00000000600322bef00342bef002e2bef003b
:101dc000302bef00000006000380d2004200ae007e
:101dd000000006008059800001002800010060001a
:101de0002eabee0030abee002e2bec0001003a00e3
:101df000302bec00282bec00300bb4000000060068
:101e0000348bd6004200ae0000000600a0598000ce
:101e1000010028000100600032abee0034abee00a0
:101e2000322bec0001003a00342bec00282bec00a4
:101e3000340bb400000006003a2bef003c2bef00ff
:101e40003e2bef00402bef00422bef00442bef0026
:101e5000462bef00482bef004a2bef004c2bef00f6
:101e60004e2bef00000006000000eb00000778009a
:101e70000c000900002f78000007eb0000000600ae
:101e8000704b8000310020000180e7002000370007
:101e900000418000410620003929af0001004000c8
:101ea0003929ae0001005000c14420000180e60045
:101eb0003929a90041bb2f000100e6003929a800fb
:101ec00000418800505888003949af002428ec00b0
:101ed0003949ae002428ed0020418000610920002e
:101ee0000180e6003949a900210320000100e60035
:101ef0003949a8008080eb0000f0a6008000eb00cc
:101f00000002020000000000b1478800c0478800be
:101f1000a1538000b053800003122400020020006f
:101f20005602020000000000fe0302000000000054
:101f300002a02000015020000180e60002005000b5
:101f4000c0538800115880002058800003122400dc
:101f5000020020005602020000000000fe03020002
:101f60000000000002a02000015020000180e600d7
:101f7000020050003058880030588000734b8000b9
:101f8000320020000218e70050588000725880008c
:101f90007058880002005000800178000150200035
:101fa00002a020000180e600820150008100ea00ca
:101fb0000100e60082014000a34e880093428800a1
:101fc000c053800031588000734b800032002000e5
:101fd0000218e700515880000218e7000000eb00eb
:101fe00001005000800178000150200002a0200074
:101ff0000180e600820150008100ea000100e60055
:1020000082014000a4002000110009008401d800d2
:102010001041880003007800022820000298e600a2
:10202000020078000201ea000218e60002007800cf
:102030007054880080428800705480000114200091
:102040000180e6007829ef000180e60010003700eb
:102050008100ea000100e6007829ef000100e600b7
:102060000b00370070548000c14b8000010040001d
:1020700080017800429c20000298e600020078006f
:102080000201ea000218e60002007800c04b880056
:10209000705480008000eb0000f0a7008080eb000f
:1020a0000002020000000000a33f24000200200004
:1020b000be02020000000000d3528000e252800005
:1020c0005602020000000000214f8800304f8800b7
:1020d000a04e80008000eb0000f0a7008080eb00a5
:1020e0000002020000000000831c24000200200007
:1020f000be02020000000000f35280000253800084
:102100005602020000000000414f8800504f880036
:10211000c04b80008000eb0000f0a7008080eb0047
:102120000002020000000000c3612400020024003d
:10213000be02020000000000135380002253800002
:102140005602020000000000614f8800704f8800b6
:10215000234f8000324f8000440302000000000043
:10216000434f8000524f80004203020000000000f5
:102170003869af0001f0a200fe0302000000000079
:1021800070428800b249800002004000800178005f
:10219000b1498000c10bb000b2498000c20bb10050
:1021a0000180e600810178000200e60082017800eb
:1021b000b34b880000f0a7000000ea008000eb00ad
:1021c0000002020000000000831c24000200200026
:1021d000be020200000000007353800082538000a2
:1021e0005602020000000000c14f8800d04f880056
:1021f000f157800000588000b3478000b24780004c
:10220000744b8000350020000520e70002003700f5
:1022100093478000a24780004203020000000000b4
:10222000d14e8800e04e8800fe030200000000004e
:10223000e24980000280e600040037000201ea0063
:102240000280e6000500370039003700e14f8000ca
:10225000f04f8000d14e8800e04e8800d1478000ca
:10226000e0478000831c240002002000be02020020
:1022700000000000535380006253800056020200a9
:1022800000000000a14f8800b04f8800d14e8000b0
:10229000e04e80008324240002002000be020200e1
:1022a00000000000335380004253800056020200b9
:1022b00000000000814f8800904f8800a34f8000ed
:1022c000b44f80004203020000000000c34f8000b2
:1022d000d24f800044030200000000003809af0024
:1022e00001f0a200fe03020000000000224a80006c
:1022f0000200400080017800214a8000c10bb0003c
:10230000224a8000c20bb1000180e6008101780002
:102310000200e60082017800834b8800404a80007a
:10232000904b8800304a8000a04b880000000600d7
:10233000204a8000804b880040498000904b8800f4
:10234000304a8000a04b88000000060022212000b7
:10235000604380000200e600624388004043800042
:102360000200e60042438800804380000200e6004d
:1023700082438800a04380000200e600a243880058
:10238000f2552000604380000280e600624388002e
:10239000404380000280e600424388008043800082
:1023a0000280e60082438800a04380000280e600ad
:1023b000a24388000729af000700370010c9ae000c
:1023c000050037000e49af0010c9a9000000eb005e
:1023d0000e49af008041880080418000310020001c
:1023e0000100e6000400370090418000e100200079
:1023f0000100e70000000600704b80002100200073
:102400000180e600020037000649a9000669a9001c
:102410000800fc00704b8000410020000180e600b5
:10242000070037000000780005003300006001005d
:10243000030037002b0037003a003700390037001f
:1024400038a9a9000e49ae000d0037000f00fc00ae
:1024500021498000f1478800304980008100400018
:1024600001488800404980008100400011488800f0
:10247000504980008100400021488800000006008b
:1024800038a9a90010c9af00420037000c48af00be
:10249000eeff37001400fc0041438000f147880044
:1024a0000001eb00604380000200e600304980003c
:1024b0008100400001488800804380000200e6005f
:1024c000404980008100400011488800a0438000fe
:1024d0000200e60050498000810040002148880049
:1024e000000006000e49ae00e5ff370038a9a8003d
:1024f0000f00fc00814b8000f1478800a04b80005a
:102500008100400001488800904b8000810040001d
:1025100011488800b04b80008100400021488800ad
:10252000000006000e49af00c5ff370010c9af001c
:10253000180037001a00fc00814b80000669ae00cd
:1025400041438000f14788000001eb0060438000b8
:102550000200e60030498000810040000148880008
:10256000804380000200e600404980008100400076
:1025700011488800b04b80000649ae00a04380009f
:102580000200e60050498000810040002148880098
:10259000000006000f00fc00e1438000f1478800c6
:1025a000f043800081004000014888000044800022
:1025b00081004000114888001044800081004000e4
:1025c0002148880000000600104980000000e0005b
:1025d00004003200d15380000e09a9000008e60073
:1025e0000e09a800a04880000000e00004003200ae
:1025f000c15280000e29a9000008e6000e29a8009b
:10260000e4488000a50020000520b900e1468000d4
:102610000e89a9000008e6000e89a800f146800096
:10262000c01220000008e6000400370040422000ed
:102630000ea9a9000008e6000ea9a8001a09e200e8
:102640000f003200d4488000431f20000320b9004f
:1026500033548000425480000ec9a9000198e6005e
:1026600001003700060037000118e70002003700bc
:102670000ec9a800020037000090e6000ec9a800ad
:10268000c0488000017d20000102b9008000eb00fd
:102690004206200011000900422ad800224780008b
:1026a00002034000c0488000410620000102b9003a
:1026b0000ee9a90004b0e6000ee9a8001009ae007a
:1026c0000000060010478000c11220000180e600d3
:1026d00010a9a9000c68af000e003700d05380008d
:1026e000a10020001029af00610020000100e600d9
:1026f0000000060070528000410120001029af0048
:10270000110420000100e600000006000c68a8008b
:1027100010a9a900d0538000510020001029af005b
:10272000310020000180e6000000060070528000a9
:10273000410120001029af00110420000180e600b3
:102740000000060010a9a8000c68a90000000600ff
:102750000e49af001c28ef001c28ec00e14080006f
:10276000900020000008e60044003700a000200090
:10277000e0408800704b8000210020000180e700cd
:102780007829ef0030438000c10d20000180e60071
:102790003a00370020448000c10d20000180e6008f
:1027a0003600370020448000010520000100e600cb
:1027b0003200370030438000910b20000100e6001a
:1027c000750037003808e20006003a002044800017
:1027d000910b20000180e6002a0037003828ec0029
:1027e000280037003628ef003828ec00c041800070
:1027f000510020000100e600220037003028ec00e4
:10280000704b8000110020000180e60006003a00b5
:1028100010c9a90080418000410020000180e6002d
:102820003028ef0015003700804180005100200063
:102830000180e6003028ef0010c9a9004100200007
:102840000100e70010c9a8000100e7000729a9005e
:10285000410020000180e70008003700404380006d
:10286000e043880060438000f0438800804380009c
:1028700000448800a0438000104488003628ef0000
:102880003828ef00304380002044880010c9ae0093
:10289000000006000e49af00000006000709a8006e
:1028a000e0438000e003b000414380000088e60080
:1028b00015003700e0438000e003b1004143800091
:1028c0000008e6001900370010448000e003b00063
:1028d000a14380000088e6001d00370010448000fe
:1028e000e003b100a14380000008e60021003700aa
:1028f0002828ef002a28ef002c28ef002e28ef00d0
:102900000709a900000006002828ec0040418000cb
:10291000e10120000180e600800037002a28ef0056
:102920002c28ef002e28ef00000006002a28ec00db
:1029300050418000e10120000180e6009300370053
:102940002828ef002c28ef002e28ef0000000600ba
:102950002c28ec0060418000e10120000180e600ad
:102960005c0337002828ef002a28ef002e28ef000c
:10297000000006002e28ec0070418000e1012000dc
:102980000180e600150337002828ef002a28ef0011
:102990002c28ef00000006003828ef0010c9af0017
:1029a000b6ff370030438000710820000180e60048
:1029b000b2ff37003608e20006003a0020448000eb
:1029c000710820000100e600acff37003628ec005b
:1029d000acff370030438000a10520000100e60075
:1029e000a6ff37003628ec00b041800051002000df
:1029f0000100e600a3ff37008429ec00204c800092
:102a0000310020000180e6008429ef007829ef00e2
:102a1000b0498000b04b88000649a9000669a900aa
:102a2000204c8000110020000100e7000649a800aa
:102a3000210020000100e7000669a8000689ae0019
:102a40000649a90006a9ae000669a900704b8000de
:102a5000210020000180e60088ff37000649a90018
:102a60000669a90085ff37001042800001428000fe
:102a70000008e700000006001069a9004208e20013
:102a80005c003a0000428000410920000180e7001c
:102a90000d00370010c9af0010c9a9000609a90030
:102aa0000629a9008629ef008829ef008a29ef006e
:102ab0003028ec0080418000510020000100e70038
:102ac0003028ef004b00370080418000e4006800b0
:102ad00048003a0000428000010920000180e70020
:102ae000170037000609a90010c9af000b00370016
:102af0008609e20043003a008809e20025013a0015
:102b00008a09e20094013a003228ed0039003b00c6
:102b1000d001200090418800360037002a28ef00bd
:102b20002828ef002c28ef002e28ef003428ed0095
:102b300030003b0020012000a04188002d0037001c
:102b400000428000110920000180e70019003700d1
:102b50000609a90010c9af000c0037008609e20081
:102b60009a003a008809e200f7013a008a09e20077
:102b700043023a003228ec0090418000e10120003d
:102b80000100e7003228ef001a0037002a28ef0082
:102b90002828ef002c28ef002e28ef003428ec0026
:102ba000a0418000310120000180e6003428ef00c0
:102bb0001000370000428000210920000180e7005a
:102bc0000400370010c9af00840237003404370016
:102bd0000800370000428000310920000180e70032
:102be0000400370010c9af00ba023700870437006d
:102bf000000037000709a900004280001042880049
:102c000000000600304c8000110020000180e70029
:102c10000f0037005829ec00c04a8000c105200091
:102c2000020320000180e600c24a8800110420004f
:102c30000180e600efff3700910320000100e6006d
:102c4000ecff370012042000c24a8800e9ff370079
:102c5000210020000180e7000f0037005a29ec0016
:102c6000d04a8000c1052000020320000180e60058
:102c7000d24a8800110420000180e600ddff370001
:102c8000910320000100e600daff37001204200063
:102c9000d24a8800d7ff3700310020000180e700ca
:102ca0000f0037005c29ec00e04a8000c1052000dd
:102cb000020320000180e600e24a8800110420009f
:102cc0000180e600cbff3700910320000100e60001
:102cd000c8ff370012042000e24a8800c5ff370011
:102ce000410020000180e7000f0037005e29ec0062
:102cf000f04a8000c1052000020320000180e600a8
:102d0000f24a8800110420000180e600b9ff370074
:102d1000910320000100e600b6ff370012042000f6
:102d2000f24a8800b3ff3700510020000180e7001d
:102d30000f0037006029ec00004b8000c105200027
:102d4000020320000180e600024b880011042000ed
:102d50000180e600a7ff3700910320000100e60094
:102d6000a4ff370012042000024b8800a1ff3700a7
:102d7000610020000180e7000f0037006229ec00ad
:102d8000104b8000c1052000020320000180e600f6
:102d9000124b8800110420000180e60095ff3700e7
:102da000910320000100e60092ff3700120420008a
:102db000124b88008fff3700710020000180e70070
:102dc0008cff370038c9aa008aff3700304c8000da
:102dd000110020000180e7000f0037005829ed00a6
:102de000c04a8000f1022000b20520000100e60088
:102df000c24a8800910320000100e6007dff3700f1
:102e0000110420000180e6007aff370092032000c1
:102e1000c24a880077ff3700210020000180e700c8
:102e20000f0037005a29ed00d04a8000f10220003f
:102e3000b20520000100e600d24a8800910320007c
:102e40000100e6006bff3700110420000180e6005e
:102e500068ff370092032000d24a880065ff3700e0
:102e6000310020000180e7000f0037005c29ed00f1
:102e7000e04a8000f1022000b20520000100e600d7
:102e8000e24a8800910320000100e60059ff370064
:102e9000110420000180e60056ff37009203200055
:102ea000e24a880053ff3700410020000180e7001c
:102eb0000f0037005e29ed00f04a8000f10220008b
:102ec000b20520000100e600f24a880091032000cc
:102ed0000100e60047ff3700110420000180e600f2
:102ee00044ff370092032000f24a880041ff370078
:102ef000510020000180e7000f0037006029ed003d
:102f0000004b8000f1022000b20520000100e60025
:102f1000024b8800910320000100e60035ff3700d6
:102f2000110420000180e60032ff370092032000e8
:102f3000024b88002fff3700610020000180e7006e
:102f40000f0037006229ed00104b8000f1022000d5
:102f5000b20520000100e600124b8800910320001a
:102f60000100e60023ff3700110420000180e60085
:102f700020ff370092032000124b88001dff37000e
:102f8000710020000180e7001aff370038c9aa004d
:102f900018ff3700404c8000110020000180e7003e
:102fa000060037009a29ec00a1002000d04c8000d8
:102fb0000180e6009a29ef004b003700404c80006a
:102fc000210020000180e700060037009c29ec006a
:102fd000a1002000e04c80000180e6009c29ef0069
:102fe00041003700404c8000310020000180e700a4
:102ff000060037009e29ec00a1002000f04c800064
:103000000180e6009e29ef0037003700404c800029
:10301000410020000180e70006003700a029ec00f5
:10302000a1002000004d80000180e600a029ef00f3
:103030002d003700404c8000510020000180e70047
:1030400006003700a229ec00a1002000104d8000ee
:103050000180e600a229ef0023003700404c8000e9
:10306000610020000180e70006003700a429ec0081
:10307000a1002000204d80000180e600a429ef007f
:1030800019003700404c8000710020000180e700eb
:1030900006003700a629ec00a1002000304d80007a
:1030a0000180e600a629ef000f003700404c8000a9
:1030b000810020000180e70006003700a829ec000d
:1030c000a1002000404d80000180e600a829ef000b
:1030d00005003700404c8000910020000180e7008f
:1030e000c4fe3700ac09aa00604d8000d0598800aa
:1030f000a0992000c1b32000b0187800b018780063
:10310000b0187800b0187800b0187800b0187800bf
:10311000b0187800b0187800700020009c0e0200f3
:103120000000000081598000414b880070598000e8
:10313000304b88000002020000000000a3c52400fc
:10314000920e2900be02020000000000a14c88007f
:10315000904c8800a7fe3700504c800011002000e2
:103160000180e70006003700ae29ec0021002000b6
:10317000704d80000180e600ae29ef005500370059
:10318000504c8000210020000180e700060037003d
:10319000b029ec00a1002000804d80000180e600f5
:1031a000b029ef004b003700504c80003100200068
:1031b0000180e70006003700b229ec00a1002000e2
:1031c000904d80000180e600b229ef0041003700f9
:1031d000504c8000410020000180e70006003700cd
:1031e000b429ec00a1002000a04d80000180e60081
:1031f000b429ef0037003700504c80005100200008
:103200000180e70006003700b629ec00a10020008d
:10321000b04d80000180e600b629ef002d00370098
:10322000504c8000610020000180e700060037005c
:10323000b829ec00a1002000c04d80000180e6000c
:10324000b829ef0023003700504c800071002000a7
:103250000180e70006003700ba29ec00a100200039
:10326000d04d80000180e600ba29ef001900370038
:10327000504c8000810020000180e70006003700ec
:10328000bc29ec00a1002000e04d80000180e60098
:10329000bc29ef000f003700504c80009100200047
:1032a0000180e70006003700be29ec00a1002000e5
:1032b000f04d80000180e600be29ef0005003700d8
:1032c000504c8000a10020000180e70049fe37003b
:1032d000c009aa00004e8000d0598800e09a200062
:1032e000c1b32000b0187800b0187800b01878008a
:1032f000b0187800b0187800b0187800b0187800ce
:10330000b0187800b0187800800020009c0e0200f1
:103310000000000081598000614b880070598000d6
:10332000504b88000002020000000000a3c52400ea
:10333000920e2900be02020000000000c14c88006d
:10334000b04c88002bfe3700404c8000110020005c
:103350000180e700050037009a29ed0062ff3b007d
:1033600093002000d34c88005fff3700404c800062
:10337000210020000180e700050037009c29ed00b6
:1033800059ff3b0093002000e34c880056ff3700b4
:10339000404c8000310020000180e700050037002c
:1033a0009e29ed0050ff3b0093002000f34c880065
:1033b0004dff3700404c8000410020000180e700b5
:1033c00005003700a029ed0047ff3b0093002000d7
:1033d000034d880044ff3700404c8000510020001e
:1033e0000180e70005003700a229ed003eff3b0009
:1033f00093002000134d88003bff3700404c8000b5
:10340000610020000180e70005003700a429ed00dd
:1034100035ff3b0093002000234d880032ff37002a
:10342000404c8000710020000180e700050037005b
:10343000a629ed002cff3b0093002000334d8800af
:1034400029ff3700404c8000810020000180e70008
:1034500005003700a829ed0023ff3b009300200062
:10346000434d880020ff3700404c80009100200031
:103470000180e700dffd3700ac09aa001aff370022
:10348000504c8000110020000180e700050037004b
:10349000ae29ed008fff3b0013002000734d880024
:1034a0008cff3700504c8000210020000180e70095
:1034b00005003700b029ed0086ff3b009300200097
:1034c000834d880083ff3700504c8000310020007e
:1034d0000180e70005003700b229ed007dff3b00c9
:1034e00093002000934d88007aff3700504c8000f5
:1034f000410020000180e70005003700b429ed00fd
:1035000074ff3b0093002000a34d880071ff37003b
:10351000504c8000510020000180e700050037007a
:10352000b629ed006bff3b0093002000b34d8800ef
:1035300068ff3700504c8000610020000180e700e8
:1035400005003700b829ed0062ff3b009300200022
:10355000c34d88005fff3700504c80007100200091
:103560000180e70005003700ba29ed0059ff3b0054
:1035700093002000d34d880056ff3700504c800048
:10358000810020000180e70005003700bc29ed0024
:1035900050ff3b0093002000e34d88004dff3700b3
:1035a000504c8000910020000180e70005003700aa
:1035b000be29ed0047ff3b0093002000f34d88003b
:1035c00044ff3700504c8000a10020000180e7003c
:1035d00088fd3700c009aa003eff37002a28ef0007
:1035e0002828ef002c28ef002e28ef00a0418000b3
:1035f0000000e00075003200a0418000e10068009a
:1036000078003200a0418000e200680081003200b2
:10361000a0418000e30068008a003200a0418000e1
:10362000e400680093003200a0418000e5006800db
:10363000a2003200a0418000e6006800a100320034
:10364000a0418000e7006800ae003200a041800089
:10365000e8006800b7003200a0418000e90068007f
:10366000c0003200a0418000ea006800c9003200ba
:10367000a0418000eb006800d2003200a041800031
:10368000ec006800e1003200a0418000ed0068001d
:1036900046013200a0418000ee0068005501320072
:1036a000a0418000ef00680064013200a04180006a
:1036b000f000680066013200a0418000f10068005f
:1036c00068013200a0418000f2006800320132003f
:1036d00048fd37002a28ef002828ef002c28ef00ab
:1036e0002e28ef00a04180000000e000c900320059
:1036f000a0418000e1006800cb003200a0418000c2
:10370000e2006800d3003200a0418000e3006800be
:10371000db003200a0418000e40068005500320068
:10372000a0418000e500680064003200a0418000f4
:10373000e6006800dd003200a0418000e70068007c
:10374000e9003200a0418000e8006800f10032008a
:10375000a0418000e9006800f9003200a04180002b
:10376000ea00680001013200a0418000eb0068001f
:1037700094003200a0418000ec006800a3003200f9
:10378000a0418000ed00680008013200a0418000e7
:10379000ee00680017013200a0418000ef006800d1
:1037a00026013200a0418000f000680028013200ac
:1037b000a0418000f100680032013200a041800089
:1037c000f2006800f40032000afd37002e29ec00f8
:1037d00071092000704980000180e6002e29ef0069
:1037e00004fd37003029ec00710920008049800079
:1037f0000180e6003029ef008000eb008049800066
:103800000002020000000000d1528800e05288004f
:10381000f8fc37003229ec00710920009049800043
:103820000180e6003229ef008000eb009049800023
:103830000002020000000000f152880000538800de
:10384000ecfc37003429ec0071092000a04980000d
:103850000180e6003429ef008000eb00a0498000e1
:10386000000202000000000011538800205388006d
:10387000e0fc3700a04380000709af00104480003f
:10388000b0498800222120000200e600b2498800e9
:10389000f25520000280e600b2498800b04980005d
:1038a000030120000300b9004306200011000900b5
:1038b0004308d80000508800cefc37003869aa00c1
:1038c000ccfc37003a29ec00910c2000d049800054
:1038d0000180e6003a29ef008000eb00d04980002b
:1038e0000002020000000000031224000200200079
:1038f0005602020000000000f157880000588800be
:10390000bcfc37003c29ec00910c2000e049800011
:103910000180e6003c29ef008000eb00e0498000d8
:103920000002020000000000e14f8800f04f880014
:10393000b0fc37003e29ec0071092000f0498000fe
:103940000180e6003e29ef008000eb00f049800096
:10395000000202000000000031538800405388003c
:10396000a4fc37004029ec0071092000004a8000c7
:103970000180e6004029ef008000eb00004a800053
:1039800000020200000000005153880060538800cc
:1039900098fc37004229ec0071092000104a800091
:1039a0000180e6004229ef008000eb00104a800011
:1039b000000202000000000071538800805388005c
:1039c0008cfc3700404380000709af00e0438000d3
:1039d000204a8800222120000200e600224a8800b6
:1039e000f25520000280e600224a8800204a80002a
:1039f000030120000300b900430620001100090064
:103a00004308d800105088007afc37003809aa0013
:103a100078fc37002e29ed0002003b0063092000ee
:103a20007349880073fc37003029ed0002003b0029
:103a300063092000834988008000eb0080498000f2
:103a40000002020000000000d1528800e05288000d
:103a500068fc37003229ed0002003b0063092000ba
:103a6000934988008000eb0090498000000202002a
:103a700000000000f1528800005388005dfc370010
:103a80003429ed0002003b0063092000a3498800af
:103a90008000eb00a049800000020200000000004e
:103aa000115388002053880052fc37003a29ed005a
:103ab00002003b00830c2000d34988008000eb000b
:103ac000d049800000020200000000000312240020
:103ad000020020005602020000000000f15788009a
:103ae0000058880043fc37003c29ed0002003b00f1
:103af000830c2000e34988008000eb00e04980004f
:103b00000002020000000000e14f8800f04f880032
:103b100038fc37003e29ed0002003b00630920001d
:103b2000f34988008000eb00f049800000020200a9
:103b30000000000031538800405388002dfc3700fe
:103b40004029ed0002003b0063092000034a880081
:103b50008000eb00004a800000020200000000002c
:103b6000515388006053880022fc37004229ed0041
:103b700002003b0063092000134a88008000eb002c
:103b8000104a80000002020000000000715388000b
:103b90008053880017fc37000709af0015fc370079
:103ba0000729a90010c9a90012fc37008043800032
:103bb0000709af0000448000404a8800222120000d
:103bc0000200e600424a8800f25520000280e6002a
:103bd000424a8800404a8000030120000300b900e7
:103be00043062000110009004308d8002050880037
:103bf00000fc3700604380000709af00f0438000fd
:103c0000304a8800222120000200e600324a880063
:103c1000f25520000280e600324a8800304a8000d7
:103c2000030120000300b900430620001100090031
:103c30004308d80030508800eefb37000689aa0000
:103c400038e9a9000689af0038e9a800e9fb370088
:103c500006a9aa003909a90006a9af003909a800d8
:103c6000e4fb37000709af00e2fb37006e29ec00e8
:103c7000704b8000410020000180e6006e29ef00bb
:103c8000dcfb37000709af00dafb37006e29ed00d7
:103c9000d8fb3b0030002000704b8800d5fb37007c
:103ca000904180000000e000b701320090418000a8
:103cb000e1006800b300320090418000e20068003b
:103cc000bb00320090418000e3006800c300320076
:103cd00090418000e4006800c10032009041800003
:103ce000e5006800c900320090418000e6006800ed
:103cf000d100320090418000e7006800d900320016
:103d000090418000e8006800e400320090418000ab
:103d1000e9006800ec00320090418000ea00680091
:103d20004f01320090418000eb0068004e013200ec
:103d300090418000ec0068005d01320090418000fd
:103d4000ed0068006601320090418000ee006800de
:103d50008401320090418000ef006800860032004c
:103d600090418000f00068004101320090418000e5
:103d7000f1006800e200320090418000f20068002b
:103d8000ef00320090418000f3006800fc00320038
:103d900090418000f40068000901320090418000e9
:103da000f50068005901320090418000f60068007b
:103db0005c01320090418000f70068001801320079
:103dc00090418000f80068001701320090418000a7
:103dd000f90068001601320090418000fa00680086
:103de0001501320090418000fb0068001401320090
:103df00090418000fc006800130132009041800077
:103e0000fd006800120132007afb3700904180000b
:103e10000000e0005c01320090418000e100680099
:103e20005e00320090418000e200680066003200cf
:103e300090418000e30068006800320090418000fb
:103e4000e40068006c00320090418000e5006800ea
:103e50007400320090418000e60068007c0032006f
:103e600090418000e70068008500320090418000aa
:103e7000e80068008f00320090418000e90068008f
:103e80009800320090418000ea006800f40032009f
:103e900090418000eb006800f30032009041800008
:103ea000ec0068000901320090418000ed006800dc
:103eb0001101320090418000ee00680029013200bb
:103ec00090418000ef0068002b003200904180009c
:103ed000f0006800e600320090418000f1006800c8
:103ee0008700320090418000f200680094003200a8
:103ef00090418000f3006800a100320090418000f2
:103f0000f4006800ae00320090418000f5006800c7
:103f10000a01320090418000f60068000c01320076
:103f200090418000f7006800bd00320090418000a1
:103f3000f8006800bc00320090418000f900680081
:103f4000bb00320090418000fa006800ba003200e5
:103f500090418000fb006800b90032009041800071
:103f6000fc006800b800320090418000fd0068004d
:103f7000b70032001ffb37001029aa0010a9a900c2
:103f80001cfb37001229ec005106200090488000ed
:103f90000180e6001229ef0016fb37001229ed0020
:103fa00014fb3b00430620009348880011fb3700b8
:103fb0001429ec00e1022000a04880000180e60006
:103fc0001429ef000bfb37001429ed0009fb3b001f
:103fd000d3022000a348880006fb37000000fe0043
:103fe0001629ec0051002000b04880000180e60056
:103ff0001629ef00fffa37001629ed00fdfa3b0005
:1040000043002000b3488800fafa37001829ec0072
:1040100051062000c04880000180e6001829ef000a
:10402000f4fa37001829ed00f2fa3b0043062000ad
:10403000c3488800effa37001a29ec005106200027
:10404000d04880000180e6001a29ef00e9fa370025
:104050001a29ed00e7fa3b0043062000d348880008
:10406000e4fa37001c29ec00b10f2000e048800082
:10407000c30320000180e600e3488800ddfa370032
:104080001c29ed00b1032000e0488000a30f2000b0
:104090000100e600e3488800d6fa37001e29ec004c
:1040a00051062000f04880000180e6001e29ef0044
:1040b000d0fa37001e29ed00cefa3b00430620005f
:1040c000f3488800cbfa370020a9ec00f115200056
:1040d00000498000a30520000180e6000349880014
:1040e000c4fa370020a9ed009105200000498000a6
:1040f000e31520000100e60003498800bdfa3700ff
:104100004043800020498800222120000200e60070
:1041100022498800f25520000280e60022498800ea
:1041200020498000030120000300b900430620005d
:10413000110009004308d80040508800adfa37004c
:104140006043800030498800222120000200e60000
:1041500032498800f25520000280e600324988008a
:1041600030498000030120000300b900430620000d
:10417000110009004308d800505088009dfa37000c
:104180008043800040498800222120000200e60090
:1041900042498800f25520000280e600424988002a
:1041a00040498000030120000300b90043062000bd
:1041b000110009004308d800605088008dfa3700cc
:1041c000a043800050498800222120000200e60020
:1041d00052498800f25520000280e60052498800ca
:1041e00050498000030120000300b900430620006d
:1041f000110009004308d800705088007dfa37008c
:10420000d0508000804a8800e0508000904a8800aa
:1042100078fa3700f0508000a04a880075fa37001d
:104220002ca9aa0073fa37002c69aa0071fa37008a
:104230002c49aa006ffa37002c89aa006dfa3700c2
:104240002cc9a8006bfa37006409aa0069fa370084
:104250001069a8009a3802000000000065fa3700d3
:104260001089aa0063fa37002c29aa0061fa3700e6
:104270003889aa006e29ef003889ae000649a900e6
:104280003889ae000669a9003889ae0004003700fd
:104290000400fc00e09324004009880055fa370030
:1042a0000400fc00f0ff27004009880051fa3700a5
:1042b0000609a8004a29ec00f1012000504a8000bc
:1042c0000180e6004a29ed004afa37000609a800f5
:1042d0004a29ed0047fa3b004a29ec0045fa37002d
:1042e0008629ec0081002000304c80000180e6002f
:1042f0008629ef003ffa37008629ed003dfa3b00a2
:1043000073002000334c88003afa37008829ec000b
:10431000a1002000404c80000180e6008829ef00c9
:1043200034fa37008a29ec00b1002000504c80009c
:104330000180e6008a29ef002efa37008829ed0077
:104340002cfa3b0093002000434c880029fa3700e8
:104350008a29ed0027fa3b00a3002000534c880077
:1043600024fa370080438000b04a8800030120000f
:104370000300b90043062000110009004308d800db
:10438000805088001bfa37000729a80010c9a80030
:1043900040438000e043880060438000f043880091
:1043a0008043800000448800a043800010448800bf
:1043b00010fa370030428000011020000100e600b2
:1043c0001c0037008000eb0047e8af008080eb0066
:1043d00030428000000202000000000043da2300a7
:1043e000f2ff2f0056020200000000001029ae006c
:1043f00004003700fe030200000000002042880095
:1044000000000600032024000200200042030200f6
:1044100000000000e3f02300428e23005602020059
:1044200000000000fe03020000000000204288009f
:10443000000006008000eb004be8af008080eb003e
:1044400050428000000202000000000043da230016
:10445000f2ff2f0056020200000000001029af00fa
:1044600004003700fe030200000000002042880024
:104470000000060063fe230062662600560202006a
:1044800000000000fe030200000000000202200005
:1044900002004000204288000000060000020200e6
:1044a0000000000073f22300f247230056020200ce
:1044b00000000000fe0302000000000000000600f3
:1044c000f401fc00000202000000000033478000fd
:1044d0004247800042030200000000001609e2008b
:1044e0000a003200b548800061836a000a00320089
:1044f00062836a000b00320063836a000c003200a2
:104500009314240012f629000c00370093042400b1
:1045100012f6290009003700930c240012f6290036
:10452000060037006310240012a4260003003700a1
:1045300073112400f288290000003700560202009f
:104540000000000001f0a600020037008000eb0030
:104550000000eb005147880060478800fe0302001e
:10456000000000001047880001f0a700e228ef00db
:104570000100e000010032000000060012002000ef
:104580000200e600000006005147800060478000fe
:10459000937e2300424520005602020000000000e6
:1045a00001f0a700060037007347800082478000b3
:1045b0004403020000000000714788008047880023
:1045c000fe0302000000000001f0a6002047880062
:1045d000000006008000eb004feaaf008080eb0097
:1045e000705280000002020000000000810178008b
:1045f00000017800560202000000000011578800f8
:1046000020578800115480002054800000020200ce
:1046100000000000810178000001780056020200cd
:10462000000000001357800022578000440302005e
:10463000000000007a04020000000000fe030200f7
:10464000000000003154880040548800000006003b
:10465000115480002054800000020200000000007d
:1046600011578800205788008000eb004feaaf0008
:104670008080eb0070528000000202000000000009
:104680001357800022578000400402000000000001
:104690005326240012ee2200560202000000000001
:1046a000fe03020000000000c05288000000060067
:1046b0000ac8a9000ae8a9000b88a900e6c02000e2
:1046c0000b68af00e6d12000b60278007704200026
:1046d0000728e70026003700670520000728e700c5
:1046e00004003700270520000728e7004c003700aa
:1046f0002b043700b60278004705200007a8e70022
:1047000000000600b60278007704200007a8e70042
:104710000000060086c020000b68af0086d1200094
:104720009800200064000700a9bb2000980020002a
:1047300068000700480020005f0007009800200084
:104740005d000700480020005b0007008800200093
:1047500059000700480020005700070089bc2000ce
:10476000880020005b0007000ae8a800000006009f
:10477000b60278007704200007a8e70000000600d2
:10478000b60278001704200007a8e7000000060022
:1047900086c020000b68af0086d120009800200062
:1047a00045000700d800200043000700c9b52000dd
:1047b000e80020004700070049b72000480020001b
:1047c0004400070089b72000f800200041000700de
:1047d00029b92000480020003e00070069b92000e8
:1047e000480020003b000700a9b920005800200025
:1047f0003800070009ba20006800200035000700d3
:10480000a9ba200098002000320007000ac8a800ba
:104810000a28ae00000006000a28a90000000600d1
:10482000b6027800d704200007a8e70000000600c1
:10483000b60278003704200007a8e7000000060051
:1048400086c020000b68af0086d1200098002000b1
:1048500019000700d80020001700070089bf2000ba
:10486000480020001b000700b800200012000700cd
:104870004800200010000700c80020000e000700bc
:10488000480020000c000700980020000a000700e4
:10489000a800200008000700a9bf20008800200011
:1048a0000c0007000b88a8000a28ae0000000600d4
:1048b0000a28a900000006000804e900b803320035
:1048c000b6027800c702200007a8e700faff370009
:1048d000000006000804e900b1033200b6027800c7
:1048e000851c7800c702200007a8e700f9ff370001
:1048f0000000060050f50700a6bf2000c9b3200045
:10490000a0c02000905a8800082502000000000086
:104910000ba8af000000060080598000b05188004d
:1049200070598000c05188000000060042f5070061
:1049300006ba2000c9b32000e0ba2000905a8800cf
:10494000ae2402000000000070598000d0518800a1
:10495000f0518000e0518800000006000bc8a9005b
:104960003e2aef000004eb00502bef003a0ba900a9
:10497000502bec008002eb00b6027800c70220004a
:104980000728e70015003700e70220000728e700a6
:104990000f003700975a80000638e60018003700ed
:1049a000d70220000728e70006003700f7002000a4
:1049b00087836200871c78000bc8af000804e800fa
:1049c000ebff37003a0ba800502bed00e8ff370053
:1049d0000bc8a800502bed00e5ff3700502bed0071
:1049e000f8518800500be20005003200500bed003a
:1049f0009c0e0200000000000ba8a90000000600a9
:104a00002e2bef00302bef000ba8a80000000600b3
:104a1000502bef003a0ba900502bec00b6027800a7
:104a2000c70220000728e70010003700e702200037
:104a30000728e7000d003700975a80000638e60087
:104a400012003700d70220000728e70004003700d3
:104a5000f700200087836200871c7800eeff370094
:104a60003a0ba800502bed00ebff3700502bed0068
:104a7000500be20005003200500bed009c0e0200ce
:104a8000000000000ba8a900000006002e2bef007c
:104a9000302bef000ba8a80000000600e6f407008a
:104aa000a6b92000c9b3200000ba2000905a88009f
:104ab000502bef00502bec00b6027800f7002000de
:104ac00087836200871c7800c70220000728e70060
:104ad00004003700975a80000638e60001003700ce
:104ae000f4ff37008024eb00502bed00000037006e
:104af000500be2002a033200500bed009c0e020026
:104b00000000000070598000e05388001c0f020074
:104b100000000000b65c8000f50020000503630083
:104b2000e6598800000020009c0e020000000000f2
:104b300070598000f053880000000600bef40700a2
:104b400086bc2000c9b32000a0bd2000905a880078
:104b5000ae240200000000008159800070598000de
:104b60001029af0017003700f55180000500e00064
:104b70001200320061836a000d00320062836a0015
:104b80000700320063836a00010032002a00370008
:104b9000833e2000110009004308d80007003700b9
:104ba00043062000110009004308d8000300370025
:104bb000a3002000110009004308d800d05388004a
:104bc000000006000002020000000000f551800015
:104bd0000500e0001000320061836a000b00320023
:104be00062836a000600320063836a0001003200bb
:104bf00011003700834c2400020020000800370019
:104c000003322400020020000500370003182400ae
:104c10000200200002003700c3fc2300d2cc2c008d
:104c2000be02020000000000fe03020000000000bf
:104c3000d0538800000006007a2aef00000006002a
:104c40007df40700a6bb2000c9b32000c0bc200033
:104c5000905a8800ae2402000000000081598000b4
:104c6000705980000002020000000000f551800031
:104c70000500e0000f00320061836a000b00320083
:104c800062836a000600320063836a00010032001a
:104c900060003700a3472400020020000500370011
:104ca000832c24000200200002003700031224009d
:104cb00002002000be02020000000000115888001f
:104cc00020588800fe0302000000000040528800c7
:104cd000115880002058800063f3230012b6200092
:104ce0005602020000000000115888002058880079
:104cf000fe030200000000003052880000000600a1
:104d00004df40700a6ba2000c9b32000c0bb2000a4
:104d1000905a8800ae2402000000000081598000f3
:104d2000705980000002020000000000f551800070
:104d30000500e0001000320061836a000b003200c1
:104d400062836a000600320063836a000100320059
:104d50003000370073b52300c2352000080037004b
:104d600063d02300a22126000500370073ea230048
:104d700002aa2f00020037001305240082942f009e
:104d80005602020000000000515288006052880064
:104d90008352800092528000420302000000000013
:104da0001029af0004003700c3e92300f2eb200014
:104db000560202000000000091478800a0478800ca
:104dc000fe0302000000000070528800914780003e
:104dd000a0478000a3528000b2528000a1528800f8
:104de000b052880042030200000000008324240027
:104df000020020005602020000000000d147880097
:104e0000e1478800fe0302000000000050548800c3
:104e100000000600000006000a68a8000000060066
:104e2000502bef00502bec00b6027800f70020006a
:104e300087836200871c7800e70220000728e700cc
:104e400007003700c70220000728e70004003700ea
:104e5000975a80000638e60001003700f1ff37005e
:104e60008024eb00502bed00000006000a88a9000a
:104e70003a0ba900502bef00502bec00b602780043
:104e8000f700200087836200871c7800e70220007b
:104e90000728e7000a003700d70220000728e700ac
:104ea0000a000700c70220000728e7000b003700b0
:104eb000975a80000638e60001003700eeff370001
:104ec0008024eb00502bed00000006003a0ba800f8
:104ed000502bed00a9027800000006000a88a80007
:104ee00000000600502bec00b6027800f70020000e
:104ef00087836200871c7800c70220000728e7002c
:104f000004003700975a80000638e6000100370099
:104f1000f4ff37008024eb00502bed00000006006a
:104f2000c5f30700e65a8000f50020000503630082
:104f3000e6598800f65a8000f5002000050363005a
:104f4000f65988003a0ba900100020009c0e0200c0
:104f500000000000815980007059800000020200aa
:104f600000000000d15e8800c05e8800b2f3070038
:104f700009b6200039037800f5002000050363001e
:104f8000e659880039037800f50020000503630026
:104f9000f65988003903780008b42000050008009d
:104fa0000300000039037800f500200005036300ca
:104fb000061c78003a0ba900700020009c0e02002d
:104fc000000000008159800070598000000202003a
:104fd0000000000043c62400021c2e00be02020096
:104fe00000000000d35e8000c25e80004403020027
:104ff00000000000e3c8230052a32f005602020065
:105000000000000001f0a000a65b8000e504200085
:105010000628e70001f0a100115f8800005f88000a
:1050200085f30700c65b8000f500200005036300e0
:10503000e6598800d65b8000f50020000503630078
:10504000f6598800e65b8000f50020000503630048
:10505000065a88003a0ba900200020009c0e02008e
:105060000000000081598000705980000002020099
:1050700000000000d15e8800c05e88006ef307006b
:10508000e9b7200039037800f5002000050363002c
:10509000e659880039037800f50020000503630015
:1050a000f65988003903780008b42000050008008c
:1050b0000300000039037800f500200005036300b9
:1050c000061c78003a0ba900700020009c0e02001c
:1050d0000000000081598000705980000002020029
:1050e0000000000043c62400021c2e00be02020085
:1050f00000000000d35e8000c25e80004403020016
:1051000000000000e3c8230052a32f005602020053
:105110000000000001f0a000965c800075052000f2
:105120000628e70001f0a100315f8800205f8800b9
:1051300000000600f0538000010020000100e6009e
:1051400000000600e0538000310020000100e6006e
:1051500000000600da2802000000000090508000e5
:10516000f14880000100e60000000600305f80008a
:10517000b0588800205f8000a0588800105f800031
:1051800090588800005f800080588800505280004e
:105190008052880060528000905288002e2aef00d2
:1051a0002c2aef002a2aef001009a8000b08a800fb
:1051b000000006003a0ae20001003a00060037004b
:1051c000d0518000014980000180e60002003700d4
:1051d000122aec0000000600122aef000000060070
:1051e000115f8000005f8000a34c8000924c800023
:1051f0004203020000000000e4040200000000007e
:10520000030024000001eb00be02020000000000c9
:1052100081017800000178005602020000000000c1
:10522000d1568800e0568800115f8000005f800042
:10523000e804020000000000115788002057880091
:10524000f156880000578800a14c8000904c8000e7
:10525000e804020000000000f356800002578000be
:105260005602020000000000f15688000057880036
:10527000315f8000205f8000c34c8000b24c800012
:105280004203020000000000e404020000000000ed
:10529000030024000001eb00be0202000000000039
:1052a0008101780000017800560202000000000031
:1052b000f3568000025780005602020000000000f2
:1052c000d3568000e2568000440302000000000034
:1052d0007a04020000000000ec040200000000005c
:1052e000030024000001eb00560202000000000051
:1052f000d1568800e05688001029af00030037001f
:1053000023ac240062be240002003700f3b924005d
:1053100092d225005602020000000000fe030200a7
:1053200000000000714c8800804c8800d15680003d
:10533000e0568000e40402000000000013578000e3
:10534000225780005602020000000000f15688003b
:1053500000578800d1568000e0568000e804020023
:1053600000000000d1568800e0568800115f8000e0
:10537000005f8000e404020000000000d3568000bb
:10538000e25680005602020000000000d15688005c
:10539000e0568800a14c8000904c8000e40402009c
:1053a00000000000d3568000e25680004203020055
:1053b00000000000f356800002578000be02020089
:1053c00000000000d1568800e056880003f8230052
:1053d0000001eb004403020000000000d3568000ef
:1053e000e256800001f0a6000200370003f82b000f
:1053f0000001eb008300780002007800f004020056
:1054000000000000d1568800e0568800c14c8000a2
:10541000b04c8000335f8000225f800042030200b6
:1054200000000000e40402000000000001f0a600fb
:105430000b003700d1568000e05680002322240064
:1054400032982f00560202000000000031578800f9
:1054500040578800fe0302000000000010003700e3
:10546000910c2400b0fd2000d3568000e25680004d
:105470004203020000000000d1568800e056880078
:105480002322240032982f00560202000000000060
:105490003157880040578800fe03020000000000da
:1054a00032528000020050000110200000f0a600df
:1054b0008000eb0001004000604c88000000060006
:1054c000115f8000005f8000935880008258800048
:1054d0004203020000000000e4040200000000009b
:1054e000030024000001eb00be02020000000000e7
:1054f00081017800000178005602020000000000df
:10550000d1568800e0568800115f8000005f80005f
:10551000e8040200000000001157880020578800ae
:10552000f15688000057880091588000805880000c
:10553000e804020000000000f356800002578000db
:105540005602020000000000f15688000057880053
:10555000315f8000205f8000b3588000a258800037
:105560004203020000000000e4040200000000000a
:10557000030024000001eb00be0202000000000056
:10558000810178000001780056020200000000004e
:10559000f35680000257800056020200000000000f
:1055a000d3568000e2568000440302000000000051
:1055b0007a04020000000000ec0402000000000079
:1055c000030024000001eb0056020200000000006e
:1055d000d1568800e05688001029af00030037003c
:1055e00023ac240062be240002003700f3b924007b
:1055f00092d225005602020000000000fe030200c5
:10560000000000001154880020548800d15680000a
:10561000e0568000e4040200000000001357800000
:10562000225780005602020000000000f156880058
:1056300000578800d1568000e0568000e804020040
:1056400000000000d1568800e0568800115f8000fd
:10565000005f8000e404020000000000d3568000d8
:10566000e25680005602020000000000d156880079
:10567000e05688009158800080588000e4040200c1
:1056800000000000d3568000e25680004203020072
:1056900000000000f356800002578000be020200a6
:1056a00000000000d1568800e056880003f823006f
:1056b0000001eb004403020000000000d35680000c
:1056c000e256800001f0a6000200370003f82b002c
:1056d0000001eb008300780002007800f004020073
:1056e00000000000d1568800e0568800b1588000c4
:1056f000a0588000335f8000225f800042030200d8
:1057000000000000e40402000000000001f0a60018
:105710000b003700d1568000e05680002322240081
:1057200032982f005602020000000000a1538800aa
:10573000b0538800fe030200000000001000370094
:10574000910c2400b0fd2000d3568000e25680006a
:105750004203020000000000d1568800e056880095
:105760002322240032982f0056020200000000007d
:10577000a1538800b0538800fe030200000000001f
:1057800032528000020050000110200000f0a600fc
:105790008000eb00010040009053880000000600ec
:1057a00000000600115f8000005f8000a3c5240098
:1057b000920e29005602020000000000fe030200c3
:1057c00000000000515f8800405f8800315f80006a
:1057d000205f8000a3c52400920e2900560202001b
:1057e00000000000fe03020000000000715f88005e
:1057f000605f8800b1588000a0588000a3c52400d5
:10580000920e29005602020000000000fe03020072
:1058100000000000f1588800e0588800915880008e
:1058200080588000a3c52400920e29005602020071
:1058300000000000fe03020000000000d1588800b4
:10584000c058880000000600544488006544880061
:10585000764488000b68ae001e003700b45a800002
:1058600085c020000428e70013003700b511800030
:10587000051a7800b45a8800a600200006a8e700a0
:10588000070037000b48a8000b68aa0084c020005e
:105890000b68ae0084d12000b45a88002b0037007a
:1058a000c6cb200004b0e6002800370084c02000ea
:1058b000b45a880025003700b51180004602200048
:1058c00006a8e70021003700051a7800b45a8800be
:1058d0001e003700b45a800085d120000428e7005c
:1058e00013003700b5118000051a7800b45a8800fb
:1058f000a600200006a8e700070037000b48a80014
:105900000b68aa0084c020000b68ae0084d1200080
:10591000b45a88000d003700c6dc200004b0e60051
:105920000a00370084d12000b45a880007003700ed
:10593000b51180004602200006a8e70003003700ea
:10594000051a7800b45a8800000037003202af0010
:10595000c0ff3700544480006544800076448000d6
:105960003222a90087c0a900004006008460a90077
:105970000040060000a0fe00849fbe00869fbe007f
:10598000889fbe008a9fbe008c9fbe00bb01800026
:105990007b578800cb0180008b578800db0180009b
:1059a0009b578800eb018000ab578800fb0180000b
:1059b000bb5788000b028000cb5788000060fe00b8
:1059c0000e49af00d1a2aa000b28aa000b28af00f5
:1059d00001003700bb003700a611020000000000e4
:1059e000282aec004a5180004b0620000bd0e7002b
:1059f0006c003700282aef002a2aec005a51800058
:105a0000cb0320000bd0e700080037002a2aef0064
:105a10002c2aec006a518000cb0320000bd0e70059
:105a2000020037002c2aef002e2aec000b08af00f2
:105a30005c0037002e0ae2005a003a002c0ae2000d
:105a400058003a003a0020005b5180000b50e700fc
:105a5000420037004a0020005b5180000b50e700f5
:105a60003c0037005a0020005b5180000b50e700db
:105a7000180037006a0020005b5180000b50e700df
:105a8000240037007a0020005b5180000bd0e70033
:105a9000440037000e49af000c48a8000e49a90089
:105aa0000c48ae003f0037008420a9009420a900d4
:105ab00084a0a90094a0a90088a0a90098a0a9008a
:105ac00088c0a90098c0a90088e0a90098e0a900b2
:105ad000340037003342a800010020009101880003
:105ae000c19a230033000800060000000000eb000c
:105af0003140ba003302ae00feff37000a00090051
:105b000000000000a01188003302ae00feff370045
:105b10008f0037003342a800010020009101880067
:105b2000419f230011000800060000000000eb0068
:105b30003140ba003302ae00feff37000a00090010
:105b400000000000a01188003302ae00feff370005
:105b50007f00370000042000c01188003342a800f5
:105b60000100200091018800019e2300130008001d
:105b7000060000000000eb003140ba003302ae0026
:105b8000feff37000a00090000000000a011880095
:105b90003302ae00feff3700a0022000c0118800d3
:105ba0006b0037000b08af00230037002e0ae2001d
:105bb00021003a002c0ae2001f003a008200200077
:105bc000535180000218e60020003700c201200077
:105bd000535180000298e600170037008000eb0068
:105be00000478000000202000000000051478800ca
:105bf000604788003147800040478000833424009c
:105c000002002000560202000000000053478000fe
:105c10006247800044030200000000009334240027
:105c200002002000be020200000000003147880090
:105c30004047880005003700e41202000000000021
:105c40008000eb00004780001dfa0700f040800054
:105c5000110020000180e700020037006409af0056
:105c60005ffd0700f0408000210020000180e70078
:105c7000020037000b08af0011fe0700f040800063
:105c8000310020000180e70005003700704b8000e4
:105c9000110020000180e600400f0200000000001b
:105ca000f0408000410020000180e7000000370044
:105cb000f0408000510020000100e6001e28ec00aa
:105cc000230037000ae8ae000f0037000829ef0074
:105cd0009afb0700dafb0700b2fe07008000eb002a
:105ce000c0468000edf90700e04688008000eb0028
:105cf000d0468000e9f90700f0468800da2102006a
:105d0000000000000ae8a9000ac8ae000900370038
:105d10001e28ef0096240200000000005ffb070031
:105d20007ffc0700f6fb07000b08ae0001fd070033
:105d30000ac8a9000b88ae00050037000829ef004b
:105d4000ecfa070023fa070041fa07000b88a900c4
:105d50000438020000000000a81302000000000048
:105d6000341502000000000082370200000000002d
:105d700020418000734b8000320020000218e700b1
:105d80007052880010418000734b80003200200068
:105d90000218e700905388000b48af005823020018
:105da000000000000b48a9009b578000db01880021
:105db000ab578000eb018800bb578000fb018800d7
:105dc000cb5780000b0288008400a9008780a900bf
:105dd0004f06be004f05be004f04be004f03be007d
:105de0004f02be000080fe00004006009780a90020
:105df00097c0a90030448800414488002342a8008d
:105e00000a00fc0080408000410320000180e60081
:105e100038003700000078003600330000600100d1
:105e2000340037003c003700440037005100370091
:105e30005e0037006b0037007800370085003700c0
:105e4000920037009f003700ac003700b9003700e0
:105e5000c6003700d3003700e0003700ed00370000
:105e6000fa0037000701370014013700210137001d
:105e70002e0137003b01370048013700550137003c
:105e8000620137006f0137007c013700890137005c
:105e900096013700a3013700b0013700bd0137007c
:105ea000c5013700cd013700d5013700dd013700ce
:105eb000e5013700ed013700fa013700070237002e
:105ec000140237002102370028023700350237005c
:105ed000420237004e0237005b023700680237008b
:105ee00075023700810237008d02370099023700b2
:105ef000a5023700804080002011880050518000aa
:105f000020118800605180002011880070518000ad
:105f1000201188009c0237008040800020118800fa
:105f2000105280002011880020528000201188002b
:105f3000305280002011880093023700804080009a
:105f40002011880070528000f10f20000080600056
:105f5000201188007052800001f02f000080600046
:105f60000080fd0020118800a041800020118800e1
:105f7000850237008040800020118800605f80002b
:105f8000f10f20000080600020118800605f800019
:105f900001f02f00008060000080fd0020118800cb
:105fa0000054800020118800770237008040800074
:105fb00020118800705f8000f10f200000806000d9
:105fc00020118800705f800001f02f0000806000c9
:105fd0000080fd0020118800e0538000201188001f
:105fe000690237008040800020118800405f8000f7
:105ff000f10f20000080600020118800405f8000c9
:1060000001f02f00008060000080fd00201188005a
:10601000f0538000201188005b0237008040800030
:1060200020118800505f8000f10f20000080600088
:1060300020118800505f800001f02f000080600078
:106040000080fd00201188009053800020118800fe
:106050004d0237008040800020118800c058800029
:10606000f10f20000080600020118800c0588000df
:1060700001f02f00008060000080fd0020118800ea
:1060800080488000201188003f0237008040800057
:1060900020118800d0588000f10f2000008060009f
:1060a00020118800d058800001f02f00008060008f
:1060b0000080fd0020118800905080002011880091
:1060c000310237008040800020118800e0588000b5
:1060d000f10f20000080600020118800e05880004f
:1060e00001f02f00008060000080fd00201188007a
:1060f0007049800020118800230237008040800012
:1061000020118800f0588000f10f2000008060000e
:1061100020118800f058800001f02f0000806000fe
:106120000080fd002011880080418000201188003f
:10613000150237008040800020118800e046800072
:10614000f10f20000080600020118800e0468000f0
:1061500001f02f00008060000080fd002011880009
:1061600090418000201188000702370080408000a5
:106170002011880020548000f10f20000080600072
:10618000201188002054800001f02f000080600062
:106190000080fd00201188008049800020118800c7
:1061a000f90137008040800020118800d053800022
:1061b000f10f20000080600020118800d053800083
:1061c00001f02f00008060000080fd002011880099
:1061d0009049800020118800eb013700804080004a
:1061e0002011880040528000f10f200000806000e4
:1061f000201188004052800001f02f0000806000d4
:106200000080fd0020118800604980002011880076
:10621000dd01370080408000201188001047800099
:10622000f10f2000008060002011880010478000de
:1062300001f02f00008060000080fd002011880028
:106240001050800020118800cf013700804080006e
:1062500020118800f0468000f10f200000806000cf
:1062600020118800f046800001f02f0000806000bf
:106270000080fd002011880030508000201188002f
:10628000c10137008040800020118800c05180008b
:10629000f10f20000080600020118800c0518000b4
:1062a00001f02f00008060000080fd0020118800b8
:1062b0002050800020118800b3013700804080000a
:1062c00020118800b0518000f10f20000080600094
:1062d00020118800b051800001f02f000080600084
:1062e0000080fd00201188000050800020118800ef
:1062f000a50137008040800020118800d051800027
:10630000f10f20000080600020118800d051800033
:1063100001f02f00008060000080fd002011880047
:10632000e0518000201188009701370080408000f4
:106330002011880000428000f10f200000806000e2
:10634000201188000042800001f02f0000806000d2
:106350000080fd0020118800b048800020118800d6
:10636000890137008040800020118800204780008c
:10637000f10f20000080600020118800204780007d
:1063800001f02f00008060000080fd0020118800d7
:10639000e0488000201188007b01370080408000a9
:1063a0002011880010548000f10f20000080600050
:1063b000201188001054800001f02f000080600040
:1063c0000080fd0020118800d04880002011880046
:1063d0006d0137008040800020118800305480001b
:1063e000f10f2000008060002011880030548000f0
:1063f00001f02f00008060000080fd002011880067
:10640000a0488000201188005f0137008040800094
:106410002011880040548000f10f200000806000af
:10642000201188004054800001f02f00008060009f
:106430000080fd0020118800c048800020118800e5
:10644000510137008040800020118800c052800038
:10645000f10f20000080600020118800c0528000f1
:1064600001f02f00008060000080fd0020118800f6
:10647000f0488000201188004301370080408000f0
:106480002011880000498000f10f2000008060008a
:10649000201188000049800001f02f00008060007a
:1064a0000080fd00201188009048800020118800a5
:1064b0003501370080408000201188005054800052
:1064c000f10f2000008060002011880050548000ef
:1064d00001f02f00008060000080fd002011880086
:1064e000704880002011880027013700804080001c
:1064f0002011880090468000f10f2000008060008d
:10650000201188009046800001f02f00008060007c
:106510000080fd0020118800a04980002011880023
:10652000190137008040800020118800a0468000bb
:10653000f10f20000080600020118800a04680003c
:1065400001f02f00008060000080fd002011880015
:10655000c0498000201188000b0137008040800076
:1065600020118800b0468000f10f200000806000fc
:1065700020118800b046800001f02f0000806000ec
:106580000080fd0020118800e04980002011880073
:10659000fd0037008040800020118800f049800015
:1065a00020118800004a800020118800104a8000d5
:1065b00020118800f40037008040800020118800fe
:1065c0004050800020118800505080002011880029
:1065d0006050800020118800eb0037008040800070
:1065e000201188007050800020118800d049800060
:1065f00020118800504a800020118800e2003700f6
:1066000080408000201188003048800020118800e0
:10661000604a800020118800704a800020118800a4
:10662000d90037008040800020118800f0428000af
:106630002011880000438000201188002043800042
:1066400020118800d0003700804080002011880091
:1066500010438000201188008050800020118800a5
:10666000c04a800020118800c700370080408000a9
:106670002011880020428000f10f2000008060007f
:10668000201188002042800001f02f00008060006f
:106690000080fd0020118800d04a80002011880071
:1066a000b9003700804080002011880070428000cf
:1066b000f10f2000008060002011880070428000ef
:1066c00001f02f00008060000080fd002011880094
:1066d000e04a800020118800ab0037008040800035
:1066e0002011880080428000f10f200000806000af
:1066f000201188008042800001f02f00008060009f
:106700000080fd0020118800f04a800020118800e0
:106710009d0037008040800020118800904280005a
:10672000f10f20000080600020118800904280005e
:1067300001f02f00008060000080fd002011880023
:10674000004b8000201188008f00370080408000bf
:1067500020118800104b800020118800304c8000f0
:1067600020118800201188008700370080408000b9
:1067700020118800304b8000f10f20000080600065
:1067800020118800304b800001f02f000080600055
:106790000080fd0020118800404c800020118800fe
:1067a000790037008040800020118800404b800035
:1067b000f10f20000080600020118800404b800015
:1067c00001f02f00008060000080fd002011880093
:1067d000504c8000201188006b0037008040800002
:1067e00020118800504b8000f10f200000806000d5
:1067f00020118800504b800001f02f0000806000c5
:106800000080fd0020118800201188005e00370004
:106810008040800020118800604b8000f10f200034
:106820000080600020118800604b800001f02f0084
:10683000008060000080fd0020118800204b800057
:10684000201188005000370080408000201188000f
:10685000704c8000f10f2000008060002011880043
:10686000704c800001f02f00008060000080fd006f
:1068700020118800604c8000201188004200370001
:106880008040800020118800804c8000f10f2000a3
:106890000080600020118800804c800001f02f00f3
:1068a000008060000080fd0020118800704b800097
:1068b00020118800340037008040800020118800bb
:1068c000d0558000f10f200000806000201188006a
:1068d000d055800001f02f00008060000080fd0096
:1068e0002011880020118800270037008040800098
:1068f00020118800e0558000f10f2000008060002a
:1069000020118800e055800001f02f000080600019
:106910000080fd0020118800201188001a00370037
:106920008040800020118800f0558000f10f200089
:106930000080600020118800f055800001f02f00d9
:10694000008060000080fd00201188002011880078
:106950000d00370080408000201188000056800024
:10696000f10f200000806000201188000056800098
:1069700001f02f00008060000080fd0020118800e1
:1069800020118800000037001028ec0081408000b2
:10699000400320000088e6001028ef00304480000b
:1069a0004144800097c0a8008400a9009780a800f7
:1069b0000040060047458800584588006945880022
:1069c000d502af0010003700070a8000584380004e
:1069d0000838e600030037008883530047438800e7
:1069e00004003700490d2300088454008703440045
:1069f000474388004745800058458000694580002e
:106a00008420a90000400600070a80004261af0010
:106a1000fdff3700574388004745800058458000f8
:106a2000694580008420a900004006008745880051
:106a300098458800a9458800d522af00100037008e
:106a4000270a8000784380000838e60003003700fa
:106a5000888353006743880004003700490d2300f2
:106a600008845400870344006743880087458000fa
:106a700098458000a945800084a0a9000040060038
:106a8000270a80004661af00fdff3700774388008a
:106a90008745800098458000a945800084a0a90012
:106aa00000400600c7458800d8458800e9458800b1
:106ab000d542af0020003700470a8000984380008d
:106ac0000838e6000b0037008883530087438800ae
:106ad0003889ae00130037000e49a900b84a80007b
:106ae00008b8e6000e49a8000c48af000e49a900fe
:106af0000c003700490d230008845400870344002c
:106b0000874388003889ae00060037000e49a90087
:106b1000b84a800008b8e6000e49a8000c48af004b
:106b20000e49a900c7458000d8458000e94580008e
:106b300088a0a90000400600470a80004a61af0013
:106b4000fdff370097438800c7458000d845800087
:106b5000e945800088a0a90000400600f7458800ac
:106b60000846880019468800d562af00100037003b
:106b7000670a8000b84380000838e6000300370049
:106b800088835300a743880004003700490d230081
:106b90000884540087034400a7438800f745800019
:106ba000084680001946800088c0a9000040060001
:106bb000670a80004e61af00fdff3700b7438800d1
:106bc000f7458000084680001946800088c0a9006b
:106bd000004006002746880038468800494688005d
:106be000d482af002e003700870a8000d84380008f
:106bf0000838e6000300370088835300c743880045
:106c000004003700490d2300088454008703440022
:106c1000c74388003821200008b8e6000600370086
:106c20003889ae000e49a8000c48af000e49a900f3
:106c30000a29ef0015003700f85520000838e60053
:106c4000060037003889ae000e49a8000c48af0096
:106c50000e49a9000a29ef000c0037000a29ec00b0
:106c600058488000a70020003889af000200370094
:106c700007c0e6000e49a90007c0e6000a29ef0098
:106c80000c48af000e49a9002221ef0027468000e2
:106c9000384680004946800088e0a9000040060090
:106ca000870a80005261af00fdff3700d74388009c
:106cb00027468000384680004946800088e0a900c9
:106cc000004006008744880098448800a944880052
:106cd0000c08af000b0037000be8a9000c08a80057
:106ce0003c28ef003e28ef005641a9005621a8009d
:106cf0005601a800a70a80005661af00f1ff3700d7
:106d000039003700a70a8000480d230008b8e600c4
:106d100027003700c8ce220008b8e6002c00370054
:106d20000be8ae0022003700c851220008b8e60088
:106d30001f0037004813220008b8e6001300370090
:106d40004896210008b8e60019003700c85721000e
:106d50000838e600160037003e28ec003c28d70033
:106d60003d68a900c8002000f941800009c0e70083
:106d70001b003700e8418000084288002fe1a8008e
:106d80009900a9000c28a800090037003e28ec0053
:106d90003c28d7003d68a800c8002000f9418000c9
:106da00009c0e7000e003700e84180000842880073
:106db0000c08a9000be8a9003c28ef003e28ef00d2
:106dc0005641a9005621a8005601a9000600370027
:106dd0000c08a8000be8a8003c28ef003e28ef00b4
:106de0005661af00b7ff370013e1a9008500a90085
:106df0000a21ef0013e1a800874480009844800036
:106e0000a94480008900a90000400600344588009c
:106e100024002000540c8800344580008440a900e0
:106e2000004006007445880024002000840c88007f
:106e30007445800084c0a90000400600b445880065
:106e400024002000b40c8800b44580008720a900ed
:106e5000004006008740a90000400600e544880085
:106e600015488000750c880025488000a50c880016
:106e7000f5478000150c880005488000450c880007
:106e800025002000250c8800e544800084e0a9004e
:106e9000004006000c28ae00070037000c28a900af
:106ea0004028ef002fe1a9008a00a9002621ef0069
:106eb0002fe1a800004006002fe1a9008a00a900e8
:106ec0002621ef008900a9009900a80000400600d3
:106ed0000a29ef003889ae000e49a8000c48af001f
:106ee0000e49a90089e0a9000040060021e3a9009d
:106ef0002043a9008de3a90085c0a90085a0a900b1
:106f00000040060005002400b50178001251800001
:106f1000440120000410b900030040000180b000cb
:106f200053012000110009004308d80010518800c7
:106f3000d0468800b501780022518000440120002d
:106f40000410b900030040000180b000530120008c
:106f5000110009004308d80020518800004788002c
:106f6000b5017800b501780002518000440120008d
:106f70000410b900030040000180b000530120005c
:106f8000110009004308d80000518800c04688005d
:106f9000b5017800624280007410b900030040001f
:106fa0000180b00053012000110009004308d800ff
:106fb00060428800d3262000030050005042880021
:106fc000b5017800b5017800b50178004242800033
:106fd0007410b900030040000180b000530120008c
:106fe000110009004308d800404288003042880060
:106ff000b5017800b5017800b5017800b5017800d9
:1070000085a0a90000000600404380000669af008b
:10701000804b8000030120000300b90043062000dc
:10702000110009004308d800f04288006043800046
:10703000030120000300b9004306200011000900ed
:107040004308d800004388008043800003012000eb
:107050000300b90043062000110009004308d800ce
:1070600010438800a04380000649af00b04b800069
:10707000030120000300b9004306200011000900ad
:107080004308d80020438800c0438000030120004b
:107090000300b90043062000110009004308d8008e
:1070a00030438800000006000100200091018800a4
:1070b000010024001100ba00f2ff2f000201680055
:1070c00011003200d04188000208200081004100f8
:1070d000024024000288e700f6ff37000208200083
:1070e000828050003100ba00029120003100080077
:1070f000030000000000eb003100ba000019780026
:1071000000000000000006000208200082805000fd
:107110003100ba0002912000310008000300000095
:107120000000eb003100ba000019780000000000f8
:1071300000000600010020009101880001002400e9
:107140001100ba00f2ff2f000201680015003200a2
:10715000d041880002082000810041000240240044
:107160000288e700f6ff37000240200082805000ce
:107170001100ba000000e800d0418800de380200ab
:1071800000000000d241800010002400003b880075
:107190000300200093018800fe3802000000000078
:1071a0000000060010002400003b8800d24180004f
:1071b000fe38020000000000000006002004240049
:1071c000003b880003002000930188008108bb0079
:1071d0000500fc0050052000303b8800a20a20007a
:1071e000323b880061e7a8000000000000000000ba
:1071f00061e7af00feff37000000060002007800e4
:107200008008bb008098bb0002912000310008007c
:10721000040000000000eb00320078008008bb0092
:107220008098bb0000000000000000000500fc008a
:1072300050052000303b8800a10a2000313b880027
:1072400061e7a800000000000000000061e7af0057
:10725000feff3700000006000000000001000000f3
:1072600004000000070000000b0000000e000000fa
:107270001100000014000000170000001b000000b7
:107280001e00000021000000250000002800000072
:107290002b0000002f00000033000000360000002b
:1072a0003a0000003e0000004200000046000000de
:1072b0004a0000004e00000052000000570000008d
:1072c0005b00000060000000650000006b00000033
:1072d00070000000760000007c00000082000000ca
:1072e000880000008f000000970000009f00000051
:1072f000a7000000af000000b9000000c3000000bc
:10730000ce000000da000000e7000000f5000000f9
:107310000401000016010000290100003e010000e8
:10732000560100007101000091010000b70100004a
:10733000e3010000180200005a020000ad02000044
:107340001a030000af03000087040000e1050000fd
:1073500069080000270f0000245000004d54000071
:107360004b330000313400002c3000002c31000081
:107370002c3100002c3100002c3000002c3000009b
:107380002c3000002c3000002c3000002c3000008d
:107390002c3000002c3000002c3000002c3000007d
:1073a0002c3000002c3000002c3000002c3000006d
:1073b0002c3000002a320000390d00000a000000c5
:1073c000245000004d5400004b32000035310000c5
:1073d0002c35000037360000303000002a32000023
:1073e000430d00000a000000245000004d5400002e
:1073f0004b320000323000002c32000030300000f0
:107400002a320000430d00000a0000002450000052
:107410004d5400004b350000303000002c3200008d
:10742000303000002c3000002c3000002c300000e8
:107430002c3000002a310000410d00000a0000003d
:10744000245000004d5400004b3300003030000049
:107450002c320000303000002c3000002c300000b6
:107460002c3000002c3000002a310000430d0000b9
:107470000a00000024470000505600005447000056
:107480002c310000393800002e390000372c000064
:10749000542c00002c4d00002c3000002e32000037
:1074a000313300002c4e00002c3000002e33000041
:1074b000393400002c4b00002c4100002a3300001e
:1074c000440d00000a00000024470000504700005f
:1074d000474100002c3000003131000035320000ff
:1074e000382e000030300000302c00003138000011
:1074f000323700002e3100003931000030300000fa
:10750000302c00004e2c00003036000039350000d1
:10751000372e0000363600003030000030300000da
:107520002c5700002c3100002c3700002c300000bc
:107530002e390000382c00002d310000382e0000bc
:1075400033310000392c00004d2c00003137000091
:107550002e380000303600002c4d00002c2c00008e
:107560002a360000460d00000a00000024470000f3
:10757000505200004d4300002c3000003533000015
:1075800037340000302e000030300000302c000076
:10759000412c000032350000303300002e36000050
:1075a00033310000392c00004e2c00003132000035
:1075b00031330000362e0000303000003939000031
:1075c0002c4500002c3200002e360000392c000023
:1075d000373900002e360000352c00003130000015
:1075e00030310000303600002c2c00002c4100000f
:0c75f0002a350000330d00000a000000e6
:020000040000fa
:0200000401f009
:04000800fdff0000f8
:020000040000fa
:0200000401f009
:04000c0078ff000079
:020000040000fa
:0200000401f009
:040010007dff000070
:020000040000fa
:0200000401f009
:04001400e7ff000002
:020000040000fa
:0200000401f009
:04001800fcff0000e9
:020000040000fa
:100008000c3b00000c3b00000c3b00000c3b0000cc
:100018000c3b00000c3b00000c3b00000c3b0000bc
:10002800f62e0000da340000063700000c3b000012
:100038000c3b000016350000123700002e37000078
:100048000c3b00000c3b00000c3b00000c3b00008c
:100058000c3b00000c3b0000763700000c3b000016
:100068000c3b00000c3b00000c3b00000c3b00006c
:100078000c3b00000c3b00000c3b00000c3b00005c
:100088000c3b00001e3700002a3700000c3b000024
:10009800ba2c00000c3b0000242c00000c3b000094
:1000a8000c3b00000c3b00000c3b00000c3b00002c
:1000b8000c3b000052350000ae350000ea35000068
:1000c800623600000c3b00000c3b00000c3b0000bb
:1000d8000c3b00000c3b00000c3b000068370000a4
:1000e8004a3700000c3b00000c3b00000c3b0000b2
:1000f8000c3b00000c3b00000c3b00000c3b0000dc
:100108000c3b00000c3b00000c3b00000c3b0000cb
:100118000c3b00000c3b00000c3b00000c3b0000bb
:100128000c3b00000c3b00000c3b00000c3b0000ab
:100138000c3b00000c3b00000c3b00000c3b00009b
:100148000c3b00000c3b00000c3b00000c3b00008b
:100158000c3b00000c3b00000c3b00000c3b00007b
:100168000c3b00000c3b00000c3b00000c3b00006b
:100178000c3b00000c3b00000c3b00000c3b00005b
:100188000c3b00000c3b00000c3b00000c3b00004b
:100198000c3b00000c3b00000c3b00000c3b00003b
:1001a8000c3b00000c3b00000c3b00000c3b00002b
:1001b8000c3b00000c3b00000c3b00000c3b00001b
:1001c8000c3b00000c3b00000c3b00000c3b00000b
:1001d8000c3b00000c3b00000c3b00000c3b0000fb
:1001e8000c3b00000c3b00000c3b00000c3b0000eb
:0801f8000c3b00000c3b000071
:020000040000fa
:100208000c3b00000c3b00000c3b00000c3b0000ca
:100218000c3b00000c3b00000c3b00000c3b0000ba
:10022800f62e0000da340000063700000c3b000010
:100238000c3b000016350000123700002e37000076
:100248000c3b00000c3b00000c3b00000c3b00008a
:100258000c3b00000c3b0000763700000c3b000014
:100268000c3b00000c3b00000c3b00000c3b00006a
:100278000c3b00000c3b00000c3b00000c3b00005a
:100288000c3b00001e3700002a3700000c3b000022
:10029800ba2c00000c3b0000242c00000c3b000092
:1002a8000c3b00000c3b00000c3b00000c3b00002a
:1002b8000c3b000052350000ae350000ea35000066
:1002c800623600000c3b00000c3b00000c3b0000b9
:1002d8000c3b00000c3b00000c3b000068370000a2
:1002e8004a3700000c3b00000c3b00000c3b0000b0
:1002f8000c3b00000c3b00000c3b00000c3b0000da
:100308000c3b00000c3b00000c3b00000c3b0000c9
:100318000c3b00000c3b00000c3b00000c3b0000b9
:100328000c3b00000c3b00000c3b00000c3b0000a9
:100338000c3b00000c3b00000c3b00000c3b000099
:100348000c3b00000c3b00000c3b00000c3b000089
:100358000c3b00000c3b00000c3b00000c3b000079
:100368000c3b00000c3b00000c3b00000c3b000069
:100378000c3b00000c3b00000c3b00000c3b000059
:100388000c3b00000c3b00000c3b00000c3b000049
:100398000c3b00000c3b00000c3b00000c3b000039
:1003a8000c3b00000c3b00000c3b00000c3b000029
:1003b8000c3b00000c3b00000c3b00000c3b000019
:1003c8000c3b00000c3b00000c3b00000c3b000009
:1003d8000c3b00000c3b00000c3b00000c3b0000f9
:1003e8000c3b00000c3b00000c3b00000c3b0000e9
:0803f8000c3b00000c3b00006f
:020000040000fa
:1078000000800000000000000f0000002d000000bc
:1078100001000000160000000000000069000000e8
:10782000460000008200000000000000010000008f
:1078300004000000070000000b0000000e00000024
:1078400004000000070000000b0000000e00000014
:10785000000000000100000004000000070000001c
:107860000b0000000e0000000400000007000000f4
:107870000b0000000e0000000000000001000000ee
:1078800004000000070000000b0000000e000000d4
:1078900004000000070000000b0000000e000000c4
:1078a00000000000010000000400000007000000cc
:1078b0000b0000000e0000000400000007000000a4
:1078c0000b0000000e00000000000000010000009e
:1078d00004000000070000000b0000000e00000084
:1078e00004000000070000000b0000000e00000074
:1078f000000000000100000004000000070000007c
:020000040000fa
:108000000000000000000000050000000a00000061
:1080100002000000160000000000000069000000df
:1080200064000000780000000a000000aa030000bd
:10803000aa0300002c030000aa0300007d0000003a
:10804000400000001400000028000000280000008c
:10805000aa030000000000000a0000006400000005
:10806000190000000000000000000000aa0300004a
:10807000aa0300002c03000014000000050000000b
:10808000010000001f07000047070000490700002b
:108090002005000052000000560000005b000000b8
:1080a0004f000000530000004400000000000000ea
:1080b00000000000000000000000000000000000c0
:0880c00002000000ffff0000b8
:020000040000fa
:1075fc000208000026060000000000000008000041
:0c760c0002000000000000000000000070
:020000040000fa
:047618000000fe0070
:00000001FF
